:100000001CC236C201C334C233C2B4C231C230C210
:100010002FC22EC22DC22CC22BC22AC229C2AE2090
:1000200000B0C8001040813FA1A6A83FA4D300D5CE
:10003000F0D922DA12DB208D14AF0000000000009E
:1000400000000000000000000000000000000000B0
:1000500000000000000000000000000000000000A0
:100060000000000000000000000000000000000090
:100070000000000000000000000000000000000080
:100080000000000000000000000000000000000070
:100090000000000000000000000000000000000060
:1000A0000000000000000000000000000000000050
:1000B0000000000000000000000000000000000040
:1000C00000F8F8F8D8F8F8F87000F0F8F8D8F8F870
:1000D000F8F000F8F8F8D8F8F8F83800F0F8F8D8A0
:1000E000F8F8F8F00070F8F8D8D8D8D89800F8F8F0
:1000F000F8001818F8F8F8181818000000000000A8
:100100000070F8F8D8D8D8D898001818F8F8F81867
:10011000181800F8F8F800F8F8F8F800F8F8F818E7
:10012000F8F8F8F000F8F8F80000F0F8F818F8F827
:10013000F8F00000000000000000000000000000D7
:1001400000878787808080808080878787808787F7
:10015000878780878787808787878780878787804B
:100160008787878780868686868787878380878735
:100170008780808087878780808080808080808063
:10018000808686868687878783808080878787802A
:100190008080808387878687878783808787878615
:1001A00087878783808787878080838787868787FD
:1001B00087838000000000000000000000000000B5
:1001C000000F0F0F0F0F0F0F0F0F0F0F0F0F0F0F4E
:1001D0000F0F0F0F0F0F0F0F0F0F0F0F0F0F0F0F2F
:1001E0000F0F0F0F0F0F0F0F0F0F0F0F0F0F0F0F1F
:1001F0000F0F0F0F0F0F0F0F0F0F0F0F0F0F0F0F0F
:100200000F0F0F0F0F0F0F0F0F0F0F0F0F0F0F0FFE
:100210000F0F0F0F0F0F0F0F0F0F0F0F0F0F0F0FEE
:100220000F0F0F0F0F0F0F0F0F0F0F0F0F0F0F0FDE
:100230000F0F0F0000000000000000000000000091
:100240000000FFFFFFFF0303FFFFFFFF0303FFFFAC
:10025000FFFF0000FFFFFFFF0000FFFFFFFF0000A8
:10026000FFFFFFFF00000000000000030303FFFF8B
:10027000FFFF0303030000FFFFFFFF0000FFFFFF7E
:10028000FF0000FFFFFFFF0000FFFFFFFF0000FF78
:10029000FFFFFF3333FFFFFFFF0000FFFFFFFF0003
:1002A00000FFFFFFFF0000FFFFFFFF3333330303B7
:1002B000030000000000000000000000000000003B
:1002C0000000030303030000030303030000030310
:1002D00003030000030303030303030303030000FA
:1002E000E3E3E3E36363E3E3E3E36060E0E0E3E3EA
:1002F0000303E0E0E0E06063636363600003E3E363
:10030000E3E36363636363630303E3E3E3E0606383
:10031000E3E3E3E000030303030000030303030339
:1003200003030303030000030303030303030303A3
:1003300003000000000000000000000000000000BA
:1003400000000000000000000000000000000000AD
:10035000000000000000000000000000000000009D
:100360007F7F7F7F00007F7F7F7F00007F7F7F7F99
:1003700000007F7F7F7F66666660606000007F7F31
:100380007F7F60667E7E7E7E00007F7F7F7F0606A9
:100390007F7F7F7F00000000000000000000000061
:1003A000000000000000000000000000000000004D
:1003B000000000000000000000000000000000003D
:1003C000000000000000000000000000000000002D
:1003D000000000000000000000000000000000001D
:1003E000000000000000000000000000000000000D
:1003F00000000000000000000000000000000000FD
:1004000000000000000000000000000000000000EC
:1004100000000000000000000000000000000000DC
:1004200000000000000000000000000000000000CC
:100430000000000000000000000011241FBECFE5F6
:10044000D2E0DEBFCDBF10E0A0E6B0E0ECE5F8E022
:1004500002C005900D92A23EB107D9F720E0A2EEAE
:10046000B0E001C01D92AD3EB207E1F7DED0F4C1AD
:10047000C7CD3FB7F8948091E7009091E800A09134
:10048000E900B091EA0022B708B601FE05C02F3F8F
:1004900019F00196A11DB11D3FBFBA2FA92F982FAA
:1004A0008827820F911DA11DB11DBC01CD0143E024
:1004B000660F771F881F991F4A95D1F7089520E08E
:1004C00030E090E0AC01022E01C0440F0A94EAF73C
:1004D00047FF02C0C09A01C0C098C29AC2982F5F5D
:1004E0003F4F2830310571F7C09AC29AC2980895DB
:1004F000C298C098C29AC09A0895C29AC09AC098E9
:10050000C2980895CF93C82FF8DF88E7D8DF80E03E
:10051000D6DF8C2FD4DFCF91EBCFEFDF88E7CFDFB3
:1005200080E4CDCFCF93DF93C0EB8C2FEBDF80E067
:10053000E9DF80E1E7DFF1DFD0E080E0C0DFDF5F0F
:10054000D038D9F7D5DFCF5FC73B79F7DF91CF91AF
:100550000895CF93DF93B89ABA9ACEE1D0E0FE0126
:100560008491D0DF2196F0E0CA33DF07C1F7DF9135
:10057000CF9108951F920F920FB60F9211242F93CF
:100580003F938F939F93AF93BF938091E30090919C
:10059000E400A091E500B091E6003091E20026E091
:1005A000230F2D3720F40296A11DB11D05C029E8A7
:1005B000230F0396A11DB11D2093E2008093E30059
:1005C0009093E400A093E500B093E6008091E700EB
:1005D0009091E800A091E900B091EA000196A11D78
:1005E000B11D8093E7009093E800A093E900B093D9
:1005F000EA00BF91AF919F918F913F912F910F9002
:100600000FBE0F901F9018951F920F920FB60F926A
:1006100011248F9381E08093EC00109260008F9101
:100620000F900FBE0F901F90189578948AB5826036
:100630008ABD8AB581608ABD83B7826083BF83B774
:10064000816083BF89B7826089BF80B7826080BFC5
:1006500080B7816080BF329A319A3098379A80E8AB
:1006600086BD16BC80E28BBF80E185BB88BB8091D4
:1006700060008823D9F12FEF89EF90E0215080406E
:100680009040E1F700C0000064DF4CDFC0EBFC2EBF
:10069000C0E0D0E032DF88E712DF80E010DF8F2D8E
:1006A0000EDF80E10CDF81E00ADF22DF36DF00E0D1
:1006B00010E0F801EC0FFD1FE65CFF4F8491FFDEB8
:1006C0000F5F1F4F00381105A1F7C058DF4F10DF33
:1006D000F394C11524E0D207E9F68FEF97EA21E6FB
:1006E000815090402040E1F700C0000080E886B9CA
:1006F000369A01E013E0C0E0D0E08091EC0088235E
:1007000081F1B7DE4B015C01B4E6CB2ED12CE12C9C
:10071000F12CAFDEDC01CB0188199909AA09BB09CC
:10072000883E9340A105B105A0F381E0C81AD10825
:10073000E108F10898EE890E93E0991EA11CB11C06
:10074000C114D104E104F10421F78091EB0082305F
:1007500020F48F5F8093EB0002C01092EB001092A8
:10076000EC008FEF99EF20E0815090402040E1F7BE
:1007700000C00000EEDED6DE8091EC00811167C083
:10078000E12CF12C80EB8E0DBDDE80E0BBDE80E144
:10079000B9DEC3DEC12CD12CF601EF59FF4F8081A9
:1007A00090E0A5E095958795AA95E1F78E159F05B0
:1007B00079F4808190E095958795959587958770D8
:1007C0009927202F01C0220F8A95EAF7822F01C0B6
:1007D00080E075DE8FEFC81AD80A90E8C916D104F8
:1007E000D9F686DE2FEFE21AF20A88E0E816F10465
:1007F00049F63699FECF24B185B117B9369A90E003
:10080000982F8827820F911D8430924008F4B4CF2E
:1008100020E030E040E13699FECF54B185B190E060
:10082000982F8827850F911D959587959595879584
:1008300017B9369A415079F78095F901EF59FF4F72
:1008400080832F5F3F4F2038310521F795CF2097C8
:0C08500009F453CFD5DB51CFF894FFCF53
:10085C00017F8285888B8F9295989B9EA1A4A7AAD5
:10086C00ADB0B2B5B8BBBEC0C3C6C8CBCDD0D2D468
:10087C00D7D9DBDDDFE1E3E5E7E9EAECEEEFF0F217
:10088C00F3F4F5F7F8F9F9FAFBFCFCFDFDFDFEFEBF
:10089C00FEFEFEFEFEFDFDFDFCFCFBFAF9F9F8F791
:1008AC00F5F4F3F2F0EFEEECEAE9E7E5E3E1DFDD96
:1008BC00DBD9D7D4D2D0CDCBC8C6C3C0BEBBB8B59C
:1008CC00B2B0ADAAA7A4A19E9B9895928F8B888558
:0208DC00820098
:00000001FF
